:100000000C9489020C94B1020C94B1020C94B102CC
:100010000C94B1020C94B1020C94B1020C94B10294
:100020000C94B1020C94B1020C94B1020C94B10284
:100030000C94B1020C94B1020C94B1020C94B10274
:100040000C94AA200C94B1020C948C230C94BE2323
:100050000C94B1020C94B1020C94B1020C94B10254
:100060000C94B1020C94B1022E05F105B1051D05E9
:10007000F105C205F105F1059E05F105F105F10552
:100080007705F105F1057C05F10541058D05810533
:10009000F1058A05F105F505CF05E005CC19D21962
:1000A000D819DE19E419EA19F1190A417661696C67
:1000B00061626C6520636F6D6D616E64733A0A20D6
:1000C000203C6E3E61202020202020202020202067
:1000D000202020202020202020202D2061637469F2
:1000E00076697479204C45442028303D6F66662C33
:1000F00020313D6F6E290A20203C7431303E2C3C6B
:1001000074313E2C3C74303E2C3C68756D3E63204F
:1001100020202D207365742074656D706572617484
:1001200075726520616E642068756D6964697479A3
:1001300020666F72207472616E736D69740A20207C
:100140003C6E3E64202020202020202020202020E3
:100150002020202020202020202D204445425547CB
:10016000206D6F64652028303D7375707072657303
:100170007320545820616E64206261642070616352
:100180006B657473290A20203C6E6E6E6E6E6E3E37
:100190006620202020202020202020202020202019
:1001A000202D206672657175656E63792028352073
:1001B0006B487A20737465707320652E672E203823
:1001C0003638333135290A20203C69643E2C3C699D
:1001D0006E743E2C3C6E62743E2C3C64723E692010
:1001E00020202D2073657420746865207061726111
:1001F0006D657465727320666F7220746865207413
:1002000072616E736D6974206C6F6F700A20203C90
:100210006E3E6D2020202020202020202020202025
:1002200020202020202020202D20746F67676C65FF
:10023000206D6F64652028313A2031372E323431F9
:10024000206B6270732C20323A20392E35373920DA
:100250006B6270732C20343A20382E383432206B85
:10026000627073290A20203C6E3E702020202020DE
:10027000202020202020202020202020202020207E
:100280002D2073686F7720726177207061796C6FB1
:10029000616420646174612028303D6F66662C20A3
:1002A000313D6F6E2C20323D6F6E6C7920756E641F
:1002B00065636F646564290A20203C6E3E722020CD
:1002C000202020202020202020202020202020202E
:1002D0002020202D206461746120726174652028C3
:1002E000303A2031372E323431206B6270732C203B
:1002F000313A20392E353739206B6270732C203219
:100300003A20382E383432206B627073290A20204C
:1003100062312C62322C62332C6234732020202014
:100320002020202020202020202D2073656E642096
:100330007468652070617373656420627974657395
:1003400020706C7573207468652063616C63756CD4
:1003500061746564204352430A20203C6E3E742041
:10036000202020202020202020202020202020208D
:10037000202020202D20746F67676C6520646174D5
:1003800061207261746520696E74657276616C6C4F
:100390002028303D6E6F20746F67676C652C203E9F
:1003A000303D7365636F6E6473290A20203C6E3E96
:1003B00076202020202020202020202020202020E7
:1003C0002020202020202D2076657273696F6E20FA
:1003D000616E6420636F6E66696775726174696FC0
:1003E0006E207265706F72740A20203C6E3E782019
:1003F00020202020202020202020202020202020FD
:10040000202020202D207573656420666F72207473
:10041000657374730A20203C6E3E792020202020D2
:1004200020202020202020202020202020202020CC
:100430002D2052656C61792028303D6E6F207265E9
:100440006C61792C20313D52656C61792072656355
:100450006569766564207061636B657473290A2031
:10046000203C6E3E7A2020202020202020202020AA
:10047000202020202020202020202D2031203D2041
:10048000646973706C617920616E616C797A6564FE
:10049000206672616D65206461746120696E737499
:1004A000656164206F66206E6F726D616C2064619F
:1004B00074610A0000000008000201000003040744
:1004C000000000000000000001020408102040802D
:1004D000010204081020010204081020040404048E
:1004E00004040404020202020202030303030303DE
:1004F0000000000023002600290000000000250065
:1005000028002B0000000000240027002A009D0482
:10051000EE2311241FBECFEFD8E0DEBFCDBF13E026
:10052000A0E0B1E0EEEEFFE502C005900D92A23B27
:10053000B107D9F725E0A2EBB3E001C01D92AC30C2
:10054000B207E1F715E0C2E1D5E004C02297FE0151
:100550000E94B12ACE30D107C9F70E9432240C94F0
:10056000F52F0C9400001F93CF93DF93CAEAD0E0DD
:10057000FE011491112371F01A3029F46DE08BE61D
:1005800094E00E948F24612F8BE694E00E948F24D8
:100590002196EECF8BE694E0DF91CF911F910C94E2
:1005A0009624CF93C82F80934F040E94EB178C2F73
:1005B0000E94EB176C2F8FEC93E0CF910C94E81610
:1005C000CF93DF93EC016430B1F460E08FEC93E003
:1005D0000E945915CE010E94B00B8C8345E0BE01EC
:1005E0008FEC93E00E940C1761E08FEC93E0DF91B9
:1005F000CF910C945915DF91CF9108954F925F924E
:100600006F927F92AF92BF92CF92DF92EF92FF9262
:100610000F931F93CF93DF93EC01643069F58B81C7
:10062000811107C099E5A92E93E4B92EC12CD12CD4
:1006300006C08BE6A82E85E2B82EC12CD12C2A81CB
:1006400030E0A0E6BAEE0E94B52A2B013C010E94E0
:10065000F4207B018C014981E40CF51C061D171D5B
:1006600084E6489FA001112421E0688186EB93E095
:100670000E94680861E006C06130B1F48881811190
:1006800013C060E086EB93E0DF91CF911F910F9153
:10069000FF90EF90DF90CF90BF90AF907F906F90E2
:1006A0005F904F900C94DB07DF91CF911F910F91DA
:1006B000FF90EF90DF90CF90BF90AF907F906F90C2
:1006C0005F904F900895CF92DF92EF92FF921F9329
:1006D000CF93DF93EC016430A1F51881812F8F73E4
:1006E000698170E09AE0899F600D711D112488274F
:1006F00077FD8095982F0E9402296B017C016A8109
:1007000070E080E090E00E9402292DEC3CEC4CEC83
:100710005DE30E94122A9B01AC01C701B6010E9451
:10072000FF27AB01BC0117FD70582B8186EB93E0CE
:10073000DF91CF911F91FF90EF90DF90CF900C94BD
:100740008608DF91CF911F91FF90EF90DF90CF90BF
:100750000895CF93DF9300D000D000D0CDB7DEB79F
:100760006FE071E08BE694E00E948D2462E171E01D
:100770008BE694E00E948D246EE28BE694E00E946A
:100780008F2467E271E08BE694E00E948D246DE295
:1007900071E08BE694E00E948D246FEC73E0CE0153
:1007A00001960E948F15BE016F5F7F4F8BE694E02C
:1007B0000E947F24CE0101960E94A42660E371E08E
:1007C0008BE694E00E948D2462E371E08BE694E076
:1007D0000E948D2480914C0490914D04892B99F0B6
:1007E00065E371E08BE694E00E948D2460914C04F7
:1007F00070914D044AE050E08BE694E00E949F2502
:1008000061E471E010C040910B0150910C016091C6
:100810000D0170910E012AE030E08BE694E00E9419
:100820008B256AE471E08BE694E00E948D2460E5FC
:1008300071E08BE694E00E948D248FEC93E00E949F
:10084000F116AB01BC012AE030E08BE694E00E9497
:100850008B2564E571E08BE694E00E948D246DE5C4
:100860008BE694E00E94CE2426960FB6F894DEBF65
:100870000FBECDBFDF91CF91089526E040E051EE4D
:1008800060E070E08BE694E00E942A2368EC70E060
:1008900080E090E00E94232180914F04882331F072
:1008A00069E571E08BE694E00E94BC2480914F04DE
:1008B0000E94D1021092580461E08EEC93E00E94F5
:1008C000A90B0E94F4206093460470934704809320
:1008D0004804909349048FEC93E00E94A91540913D
:1008E0000701509108016091090170910A018FEC94
:1008F00093E00E94B91440910B0150910C0160915A
:100900000D0170910E018FEC93E00E945A1460E08B
:1009100086EB93E00E94DB0761E08FEC93E00E949E
:10092000591580914F04882331F06CE971E08BE612
:1009300094E00E94BC240C94A903EF920F9322E050
:10094000E22E0AE02DE04CE06BE08FEC93E00E9499
:100950008C168EEC93E00E94630B6FEC73E086EBD9
:1009600093E00F91EF900C94BB07CF92DF92EF9240
:10097000FF920F931F93CF93DF93CDB7DEB7C15490
:10098000D1090FB6F894DEBF0FBECDBF8BE694E061
:100990000E944722892B09F438C18BE694E00E941B
:1009A0006022082F8C3269F4E091250481E08E0FDB
:1009B00080932504F0E0EA5DFB4F8091B2038083D1
:1009C00014C180ED800F8A3010F52091B203309170
:1009D000B3034091B4035091B503AAE0B0E00E9484
:1009E000C42A6053710981099109112707FD1095E7
:1009F000212F312F600F711F821F931F6093B2034D
:100A00007093B3038093B4039093B503FEC08FE952
:100A1000800F8A3108F0F2C0802F992787FD9095CA
:100A2000A92FB92FFC01E156F109EA31F10508F0CF
:100A3000D8C0EC5CFF4F0C94AF2A81E04091B20328
:100A40005091B3036091B4037091B503452B462BCD
:100A5000472B09F480E00E94D102C7C061E0809179
:100A6000B2039091B303A091B403B091B503892B65
:100A70008A2B8B2B09F460E08EEC93E00E94A90B8B
:100A8000B4C08091B2039091B303A091B403B0912C
:100A9000B50381309105A105B10581F050F0823098
:100AA0009105A105B10571F48AE892E2A0E0B0E0F9
:100AB00009C089E593E4A0E0B0E004C08BE695E2CC
:100AC000A0E0B0E080930B0190930C01A0930D0186
:100AD000B0930E0140910B0150910C0160910D01FA
:100AE00070910E018FEC93E00E945A147EC08091A9
:100AF000B2038093060179C08091B20380934A04C7
:100B000074C08091B2039091B30390934D0480938D
:100B10004C046BC00E94A90368C060912504E62FB5
:100B2000F0E0EA5DFB4F8091B20380836F5F6093DA
:100B3000250486E294E00E94E00210C06091250442
:100B4000E62FF0E0EA5DFB4F8091B20380836F5F98
:100B50006093250486E294E00E94FE021092250430
:100B600044C060912504E62FF0E0EA5DFB4F8091E0
:100B7000B20380836F5F6093250486E294E00E9455
:100B80006303ECCF4091B2035091B3036091B4037F
:100B90007091B5038FEC93E00E94B91426C021E058
:100BA0008091B2039091B303A091B403B091B503C7
:100BB000892B8A2B8B2B09F420E020934B0415C042
:100BC00021E08091B2039091B303A091B403B0915E
:100BD000B503892B8A2B8B2B09F420E020934E043C
:100BE00004C00E94A9030E94B3021092B2031092A3
:100BF000B3031092B4031092B50307C00152003240
:100C000020F40E94A9030E94B30286EB93E00E94A5
:100C1000DE07882351F062E08EEC93E00E94790BAE
:100C200061E08FEC93E00E9459158FEC93E00E94F5
:100C3000D9138FEC93E00E943F12882309F4F4C08B
:100C400060E08FEC93E00E945915BE016F5F7F4F0B
:100C50008FEC93E00E942D1280914E048823A9F01E
:100C6000CE0101960E94CB1BCE0101960E94940DED
:100C7000CE0101960E947F10CE0101960E9440098C
:100C8000CE0101960E949E1E22C080914A0461E01E
:100C9000813011F58EEC93E00E94790B8E010F5F8D
:100CA0001F4F7E0121E4E20EF11CF80161918F01DA
:100CB00040E150E08BE694E00E94982562E571E007
:100CC0008BE694E00E948D240E151F0571F78BE6CC
:100CD00094E00E949624A3C08EEC93E00E94790BCE
:100CE00080914F04882319F16FEC71E08BE694E05A
:100CF0000E948D248E010F5F1F4F7E01F1E1EF0EE8
:100D0000F11CF80161918F0140E150E08BE694E025
:100D10000E94982562E571E08BE694E00E948D24A4
:100D20000E151F0571F78BE694E00E949624CE0104
:100D300001960E94171D882331F0CE0101960E9472
:100D40006119482F49C0CE0101960E949E0E811163
:100D50003CC0CE0101960E94DE11882311F046E0CE
:100D60003BC0CE0101960E94090B811130C0CE011B
:100D700001960E9457208111F2CFCE0101960E9468
:100D80008D1F811126C080914A04823021F58E0189
:100D90000F5F1F4F7E01F1E4EF0EF11CF80161912E
:100DA0008F0140E150E08BE694E00E94982562E5D7
:100DB00071E08BE694E00E948D240E151F0571F7FB
:100DC0008BE694E00E94962406C045E005C04CE006
:100DD00003C044E001C040E080914B048823F9F057
:100DE0004423E9F060E470E080E090E022964FAFA9
:100DF00022970E94232122964FAD2297BE016F5F5A
:100E00007F4F8FEC93E00E940C1780914F04882352
:100E100031F06EEE71E08BE694E00E94BC2461E05C
:100E20008FEC93E00E94591580914C0490914D04F1
:100E3000892B09F490C00E94F4200091460410917F
:100E400047042091480430914904601771078207D4
:100E5000930740F4109246041092470410924804FD
:100E6000109249040E94F420E0914C04F0914D044A
:100E700048EE53E0E49F9001E59F300DF49F300D64
:100E80001124C0904604D0904704E0904804F090AC
:100E90004904C20ED31EE11CF11CC616D706E80693
:100EA000F90608F058C080910B0190910C01A091B7
:100EB0000D01B0910E018A38F2E29F07A105B1053C
:100EC000C1F48091060181FF05C08BE695E2A0E0A8
:100ED000B0E006C080FF29C089E593E4A0E0B0E05F
:100EE00080930B0190930C01A0930D01B0930E0120
:100EF0001CC08B3625E29207A105B10559F48091FB
:100F0000060180FDE9CF82FF10C08AE892E2A0E0EE
:100F1000B0E0E6CF89359344A105B10531F4809165
:100F2000060182FDF2CF81FDD0CF40910B0150919F
:100F30000C0160910D0170910E018FEC93E00E9405
:100F40005A140E94F42060934604709347048093DF
:100F5000480490934904CF5BDF4F0FB6F894DEBF8F
:100F60000FBECDBFDF91CF911F910F91FF90EF90FA
:100F7000DF90CF900895FC0171836083128249E570
:100F800053E460E070E04383548365837683178283
:100F9000138A1786108A118A128A80EA9FE0918745
:100FA0008087148A158A168A178A168612861386EF
:100FB000148615860895FC0162830895CF92DF920E
:100FC000EF92FF920F931F93CF93DF93CDB7DEB7CE
:100FD00061970FB6F894DEBF0FBECDBF8C01FC0148
:100FE0008281882391F00E94F420F80120853185C8
:100FF000C488D588E688F788C20ED31EE11CF11C90
:101000006C157D058E059F0510F480E052C00E948E
:10101000F420F801648B758B868B978B86858823EB
:1010200061F00E94F420F801C284D384E484F58442
:101030006C157D058E059F05C8F5F80187818A83AB
:1010400086858B831C8287859089A189B2898D834F
:101050009E83AF83B887198683898A87808191812F
:101060000E94EB166B017C01F8014381548165817C
:101070007681808191810E945A14BE01635F7F4F07
:10108000CE0101960E94B30B45E0BE01635F7F4F26
:10109000F801808191810E940C17B701A601F80127
:1010A000808191810E945A1481E003C0F801168664
:1010B000C4CF61960FB6F894DEBF0FBECDBFDF91EF
:1010C000CF911F910F91FF90EF90DF90CF900895F7
:1010D000AF92BF92CF92DF92EF92FF920F931F9346
:1010E000FC016783518740872687E286F386048761
:1010F0001587A382B482C582D6821F910F91FF907B
:10110000EF90DF90CF90BF90AF900895FC0147879C
:10111000508B618B728B238B089520E030E040E090
:10112000FC015191CF01450F2F5F3F4F2C3031050E
:10113000B9F781E0411180E008950F931F93CF9399
:10114000DF938C01EB0181E0898FF8018081888336
:10115000818189838481282F221F2227221F2D83AA
:10116000828190E0982F88273381832B9B838A8309
:10117000918581E096FF80E08E8BF8019185892F23
:10118000881F8827881F8F8B2223A1F01E821F8231
:10119000188619861A861B861C861D861E861F8643
:1011A000188A198A1A8A1B8A1C8A1D8A1C82188E20
:1011B000198E61C0F801608570E080E090E00E94C7
:1011C000022920E030E040E05FE30E94122A20E0A4
:1011D00030E040E053E40E94FF276E837F838887DE
:1011E0009987F801668170E0762F66278781682BE2
:1011F000882777FD8095982F0E9402296A877B8730
:101200008C879D87F80164816F7370E0762F662765
:101210008581682B75956795882777FD8095982F30
:101220000E9402296E877F87888B998BF8016185E0
:101230006F7370E0762F66278285682B882777FD8D
:101240008095982F0E94022920E030E048EC52E47B
:101250000E9467286A8B7B8B8C8B9D8BF801948115
:1012600081E096FF80E08C83F8018385888FC80138
:101270000E948D08898FDF91CF911F910F91089562
:10128000EF92FF920F931F93CF93DF93CDB7DEB70B
:10129000AA970FB6F894DEBF0FBECDBF7C01BE018A
:1012A0006F5F7F4F0E949D080E94F42000915004C0
:1012B000109151042091520430915304601B710B22
:1012C000820B930B9F938F937F936F9326EF31E065
:1012D0003F932F938E01055E1F4F1F930F930E9424
:1012E000142D0E94F4206093500470935104809355
:1012F000520490935304B8018BE694E00E948D242D
:101300006CEF71E08BE694E00E948D2487010FB6AC
:10131000F894DEBF0FBECDBFE12CF12CF801619136
:101320008F0140E150E08BE694E00E94982562E551
:1013300071E08BE694E00E948D24FFEFEF1AFF0A24
:101340008CE0E816F10451F766E072E08BE694E079
:101350000E948D248A8D811103C068E072E002C072
:1013600063E172E08BE694E00E948D246BE172E011
:101370008BE694E00E948D2440E150E069818BE689
:1013800094E00E94982562E571E08BE694E00E946B
:101390008D2440E150E06A818BE694E00E9498251C
:1013A0006FE172E08BE694E00E948D246B817C817A
:1013B00040E150E08BE694E00E949F2564E272E0F9
:1013C0008BE694E00E948D244F81588569857A854B
:1013D00022E030E08BE694E00E94902668E272E022
:1013E0008BE694E00E948D244B855C856D857E851F
:1013F00022E030E08BE694E00E9490266DE272E0FD
:101400008BE694E00E948D244F85588969897A89FA
:1014100022E030E08BE694E00E94902661E372E0E7
:101420008BE694E00E948D244B895C896D897E89CE
:1014300022E030E08BE694E00E94902667E372E0C1
:101440008BE694E00E948D246D8170E04AE050E0CC
:101450008BE694E00E9483256EE372E08BE694E0D5
:101460000E948D246E8170E04AE050E08BE694E0AB
:101470000E94832565E472E08BE694E00E948D244F
:101480004AE050E0698D8BE694E00E9498258BE657
:1014900094E00E949624AA960FB6F894DEBF0FBE81
:1014A000CDBFDF91CF911F910F91FF90EF900895E5
:1014B000FF920F931F93CF93DF93EC018B0163E5B2
:1014C00071E00E9412276BE472E0CE010E947B273C
:1014D000F8016381CE010E949E2762E571E0CE0192
:1014E0000E947B27F8016281CE010E949E2762E55F
:1014F00071E0CE010E947B2720E030E040E251E421
:10150000F80166817781808591850E94122A0E9468
:10151000CF28F62E672FCE010E949E2762E571E04C
:10152000CE010E947B276F2DCE010E949E2762E58F
:1015300071E0CE010E947B27F80162857385848566
:1015400095850E94CF28672FCE010E949E2762E5D5
:1015500071E0CE010E947B27F80162857385848546
:1015600095850E94D428CE010E949E2762E571E0F5
:10157000CE010E947B27F801668577858089918955
:101580000E94CF28672FCE010E949E2762E571E05E
:10159000CE010E947B27F801668577858089918935
:1015A0000E94D428CE010E949E2762E571E0CE0100
:1015B0000E947B2720E030E048EC52E4F801628989
:1015C0007389848995890E94122A0E94CF28F62E59
:1015D000672FCE010E949E2762E571E0CE010E9436
:1015E0007B276F2DCE010E949E2762E571E0CE0120
:1015F0000E947B27F8016581660F8481680FCE0108
:101600000E949E27CE01DF91CF911F910F91FF90F5
:1016100008950F931F93CF93DF93CDB7DEB7A697AF
:101620000FB6F894DEBF0FBECDBF8C0163E571E04D
:10163000CE0181960E941227F8018081853211F532
:101640008181982F9F7B9A3211F08034D9F4BE01AA
:101650006F5F7F4FC8010E949D088A8D882391F09B
:10166000BE016F5F7F4FCE014B960E94580ABE01AC
:10167000655E7F4FCE0181960E942827CE014B9652
:101680000E94A4268DA19EA1892B39F0BE016F5D19
:101690007F4F8BE694E00E94AA2411E02DA13EA189
:1016A000232B09F410E0CE0181960E94A426812FFD
:1016B000A6960FB6F894DEBF0FBECDBFDF91CF91D7
:1016C0001F910F91089521E0FC0120830895CF938D
:1016D000C62FFC018081882351F061E089E00E94DF
:1016E000AF2161E06C2789E0CF910C94E821CF9184
:1016F0000895EF92FF920F931F93CF93DF938C0186
:10170000662301F16B3008F06AE0C0E0D0E0E62E1D
:10171000F12CCE15DF05B4F461E0C8010E94670B1F
:1017200062E370E080E090E00E94232160E0C80165
:101730000E94670B62E370E080E090E00E9423214A
:101740002196E7CFDF91CF911F910F91FF90EF90FE
:101750000895FC016083611102C00C94670B089529
:1017600064E00C94D2178F929F92AF92BF92CF9267
:10177000DF92EF92FF920F931F93CF93DF938C0131
:10178000EB01FB0180E090E011920196853091051C
:10179000D9F780E98883F8018181869586958069EB
:1017A00088838181F0E48F9FC00111248983F8012F
:1017B0002281F0E22F9F90011124822B8983F8016E
:1017C0002381F0E12F9F90011124B82EB22AB98213
:1017D00020E030E040E252E4F801648175818681C6
:1017E00097810E94FF276B017C0120E030E040E2FE
:1017F00051E40E9467280E94CF28B62AB98220E0CF
:1018000030E040E85FE3C701B6010E9444294B0184
:101810005C01C701B6010E94CF28CB016AE070E0ED
:101820000E94792A24E0880F991F2A95E1F7FA800F
:10183000F82A20E030E040E251E4C501B4010E9402
:10184000122A20E030E040E05FE30E94FF270E9480
:10185000CF28F62AFA82F80121852B838085F0E8CB
:101860008F9FC0011124822B8B83CE010E94B00B6D
:101870008C83DF91CF911F910F91FF90EF90DF90BC
:10188000CF90BF90AF909F908F900895BF92CF92CE
:10189000DF92EF92FF920F931F93CF93DF938C0110
:1018A000EB0181E08B87F801F480FA86C8010E9481
:1018B000B00BF8121B861982F80180818F70F4E05A
:1018C0008F9FC0011124898330915804F801218130
:1018D000922F332311F0907C04C0929596959695A3
:1018E0009370982B9983F801808182958F708883FB
:1018F000893009F01B86F801818185FB882780F9F2
:101900008A838181829581708B83B28061816F70BF
:1019100070E080E090E00E94022920E030E048EC96
:1019200052E40E94122A20E030E0A9010E94FF2721
:101930006B017C016B2D62956F7070E080E090E030
:101940000E94022920E030E040E251E40E94122A85
:101950009B01AC01C701B6010E94FF276B017C010E
:101960006B2D6F7070E080E090E00E9402299B0177
:10197000AC01C701B6010E94FF2720E030E040E241
:1019800051E40E94672820E030E040E252E40E94E7
:10199000FE276C837D838E839F83F8019381892F3B
:1019A000881F8827881F888783818F778987DF91A1
:1019B000CF911F910F91FF90EF90DF90CF90BF904C
:1019C0000895AF92BF92CF92DF92EF92FF920F9362
:1019D0001F93CF93DF9300D000D000D0CDB7DEB7F8
:1019E0005C018B0163E571E0CE0101960E94122734
:1019F00067E572E0CE0101960E947B27F8016181C4
:101A0000CE0101960E949E2760E2CE0101960E94BF
:101A10008B27F80181858F77843610F08A3651F450
:101A2000F8018281882319F061E870E008C061E064
:101A300070E005C08D3709F042C062E870E0CE0169
:101A400001960E94CB2760E2CE0101960E948B276F
:101A500020E030E040E251E4F80164817581868144
:101A600097810E94122A20E030E04AE754E40E9465
:101A7000FF270E94D428F62E672FCE0101960E94E0
:101A80009E2760E2CE0101960E948B276F2DCE012A
:101A900001960E949E2760E2CE0101960E948B274C
:101AA000F801C480D580E680F78020E030E040E790
:101AB00052E4C701B6010E940E2A87FD06C063E505
:101AC00071E0C5010E94122719C020E030E040E219
:101AD00052ECC701B6010E946328181684F7F8017A
:101AE0006185808581116068CE0101960E949E27E4
:101AF000BE016F5F7F4FC5010E943F27CE01019657
:101B00000E94A426C50126960FB6F894DEBF0FBE2C
:101B1000CDBFDF91CF911F910F91FF90EF90DF909C
:101B2000CF90BF90AF900895EF92FF920F931F93C5
:101B3000CF93DF93CDB7DEB7A1970FB6F894DEBF92
:101B40000FBECDBF7C01BE016F5E7F4F0E94460C71
:101B50001D8E1E8E1F8E18A219A22A89FE017D9647
:101B6000CE0182963191231709F4DBC0E817F907FB
:101B7000C9F70E94F420009154041091550420915B
:101B8000560430915704601B710B820B930B9F938B
:101B90008F937F936F9386EF91E09F938F938E0146
:101BA0000F5F1F4F1F930F930E94142D0E94F4206C
:101BB0006093540470935504809356049093570493
:101BC000B8018BE694E00E948D2467E872E08BE612
:101BD00094E00E948D2487010FB6F894DEBF0FBEFB
:101BE000CDBFE12CF12CF80161918F014AE050E06A
:101BF0008BE694E00E94982562E571E08BE694E024
:101C00000E948D24FFEFEF1AFF0A85E0E816F10429
:101C100051F766E072E08BE694E00E948D248C8D93
:101C2000811107C068E072E08BE694E00E948D2489
:101C300074C063E172E08BE694E00E948D246BE156
:101C400072E08BE694E00E948D244AE050E06989BE
:101C50008BE694E00E9498256FE172E08BE694E0B9
:101C60000E948D244AE050E06A898BE694E00E944D
:101C700098256DE572E08BE694E00E948D246B89D7
:101C800070E04AE050E08BE694E00E94832567E62E
:101C900072E08BE694E00E948D246C8970E04AE04B
:101CA00050E08BE694E00E9483256FE672E08BE6BD
:101CB00094E00E948D244D895E896F89788D22E0A1
:101CC00030E08BE694E00E94902666E772E08BE6B7
:101CD00094E00E948D24698D70E04AE050E08BE62C
:101CE00094E00E94832561E872E08BE694E00E9414
:101CF0008D244AE050E06A8D8BE694E00E9498259E
:101D000065E472E08BE694E00E948D244AE050E0A6
:101D10006B8D8BE694E00E9498258BE694E00E9400
:101D20009624A1960FB6F894DEBF0FBECDBFDF910B
:101D3000CF911F910F91FF90EF9008950F931F93F4
:101D4000CF93DF93CDB7DEB768970FB6F894DEBFB9
:101D50000FBECDBF8C0163E571E0CE0143960E94BA
:101D60001227F801808182958F70893031F5BE018C
:101D70006F5F7F4FC8010E94460C8C85882391F0CD
:101D8000BE016F5F7F4FCE010D960E94E10CBE0138
:101D9000635F7F4FCE0143960E942827CE010D96A8
:101DA0000E94A4268F89988D892B39F0BE016D5E23
:101DB0007F4F8BE694E00E94AA2411E02F89388D92
:101DC000232B09F410E0CE0143960E94A426812F14
:101DD00068960FB6F894DEBF0FBECDBFDF91CF91EE
:101DE0001F910F91089565E00C94D2178F929F92E6
:101DF000AF92BF92CF92DF92EF92FF920F931F9319
:101E0000CF93DF938C01EB0181E08F87F801F580A0
:101E1000FE86C8010E94F30EF81659F080915D0409
:101E2000882331F062E972E08BE694E00E94BC24E2
:101E30001F86F80180818F708983808182958F70E1
:101E400088838B3059F080915D04882331F061EAFA
:101E500072E08BE694E00E94BC241F86F801618149
:101E600062956F70F4E66F9FB0011124882777FDAB
:101E70008095982F0E9402296B017C016A837B83E5
:101E80008C839D83F80161816F70FAE06F9FB001D0
:101E90001124882777FD8095982F0E9402299B01A5
:101EA000AC01C701B6010E94FF276B017C016A8368
:101EB0007B838C839D83F801628162956F7070E0F3
:101EC00080E090E00E9402299B01AC01C701B601AD
:101ED0000E94FF2720E030E040E05FE30E94122AEA
:101EE0006A837B838C839D83F80162816F70FAE043
:101EF0006F9FB0011124882777FD8095982F0E944D
:101F000002296B017C016E837F8388879987F801A2
:101F1000638162956F7070E080E090E00E9402291A
:101F20009B01AC01C701B6010E94FF276B017C0138
:101F30006E837F8388879987F80163816F7070E073
:101F400080E090E00E9402292DEC3CEC4CEC5DE33B
:101F50000E94122A9B01AC01C701B6010E94FF2713
:101F600020E030E040E252E40E94FE276B017C0159
:101F70006E837F8388879987F801648162956F708B
:101F800070E080E090E00E9402294B015C016A87CA
:101F90007B878C879D87F80164816F7070E080E09B
:101FA00090E00E9402292DEC3CEC4CEC5DE30E9499
:101FB000122A9B01AC01C501B4010E94FF276A8768
:101FC0007B878C879D8720E030E040E252ECC701A0
:101FD000B6010E94632887FD0AC020E030E040E798
:101FE00052E4C701B6010E940E2A1816ACF41F86EF
:101FF00080915D04882381F060EB72E08BE694E0D1
:102000000E948D244E815F816885798522E030E0D1
:102010008BE694E00E949226CA80DB80EC80FD80F3
:1020200020E030E040E050E4C701B6010E946328A0
:1020300087FD0AC020E030E046E953E4C701B6015D
:102040000E940E2A1816ACF41F8680915D04882326
:1020500081F067EC72E08BE694E00E948D244A8167
:102060005B816C817D8122E030E08BE694E00E9410
:102070009226CA84DB84EC84FD8420E030E040E0DA
:1020800050E4C701B6010E94632887FD0AC020E022
:1020900030E040E551E4C701B6010E940E2A18164F
:1020A0000CF51F8680915D048823E1F068ED72E0F5
:1020B0008BE694E00E948D244A855B856C857D8546
:1020C00022E030E08BE694E0DF91CF911F910F91F9
:1020D000FF90EF90DF90CF90BF90AF909F908F9048
:1020E0000C949226DF91CF911F910F91FF90EF906A
:1020F000DF90CF90BF90AF909F908F900895EF9218
:10210000FF920F931F93CF93DF93CDB7DEB7A097C6
:102110000FB6F894DEBF0FBECDBF7C01BE016F5E6F
:102120007F4F0E94F60E0E94F420009159041091F6
:102130005A0420915B0430915C04601B710B820B8C
:10214000930B9F938F937F936F9326EF31E03F9391
:102150002F938E010F5F1F4F1F930F930E94142D1B
:102160000E94F4206093590470935A0480935B0496
:1021700090935C04B8018BE694E00E948D246BEE92
:1021800072E08BE694E00E948D2487010FB6F894EC
:10219000DEBF0FBECDBFE12CF12CF80161918F01A4
:1021A00040E150E08BE694E00E94982562E571E002
:1021B0008BE694E00E948D24FFEFEF1AFF0A86E081
:1021C000E816F10451F766E072E08BE694E00E94B5
:1021D0008D2488A1811107C068E072E08BE694E04D
:1021E0000E948D245DC063E172E08BE694E00E9462
:1021F0008D246BE172E08BE694E00E948D244AE02E
:1022000050E069898BE694E00E9498256FE172E0C6
:102210008BE694E00E948D244AE050E06A898BE6C8
:1022200094E00E94982569EF72E08BE694E00E94AA
:102230008D244B895C896D897E8922E030E08BE6B4
:1022400094E00E9490266FE672E08BE694E00E9494
:102250008D244F89588D698D7A8D22E030E08BE690
:1022600094E00E94902661E073E08BE694E00E9487
:102270008D244B8D5C8D6D8D7E8D22E030E08BE664
:1022800094E00E94902665E472E08BE694E00E9460
:102290008D244AE050E06F8D8BE694E00E949825F3
:1022A0008BE694E00E949624A0960FB6F894DEBFC9
:1022B0000FBECDBFDF91CF911F910F91FF90EF9097
:1022C0000895FF920F931F93CF93DF93EC018B013F
:1022D00063E571E00E94122768E073E0CE010E947E
:1022E0007B27F8016181CE010E949E276FE073E099
:1022F000CE010E947B2720E030E040E251E4F8016B
:1023000062817381848195810E94122A20E030E0ED
:102310004AE754E40E94FF270E94CF28F62E672F39
:10232000CE010E949E2762E571E0CE010E947B27CC
:102330006F2DCE010E949E2762E571E0CE010E94C2
:102340007B2720E030E040E251E4F80166817781AC
:10235000808591850E94122A20E030E04AE754E40B
:102360000E94FF270E94CF28F62E672FCE010E94E1
:102370009E2762E571E0CE010E947B276F2DCE0182
:102380000E949E2762E571E0CE010E947B2720E03B
:1023900030E040E251E4F8016285738584859585DB
:1023A0000E94122A0E94CF28CE010E94CB27CE0184
:1023B000DF91CF911F910F91FF9008950F931F937D
:1023C000CF93DF93CDB7DEB76C970FB6F894DEBF2F
:1023D0000FBECDBF8C0163E571E0CE0147960E9430
:1023E0001227BE016F5F7F4FC8010E94F60E8889D9
:1023F000882391F0BE016F5F7F4FCE0141960E940E
:102400006111BE016F5E7F4FCE0147960E94282763
:10241000CE0141960E94A4268B8D9C8D892B39F08C
:10242000BE01695E7F4F8BE694E00E94AA2411E012
:102430002B8D3C8D232B09F410E0CE0147960E9492
:10244000A426812F6C960FB6F894DEBF0FBECDBFC9
:10245000DF91CF911F910F910895FC01158A108A89
:10246000FB0120E030E0DC01A20FB31F56964C9137
:1024700041932F5F3F4F20343105A9F70895FC01A8
:10248000858908950F931F93CF93DF93DC01862FE7
:1024900013966C91139770E0FB01E452FB4FE491AB
:1024A000F0E0EE0FFF1FE051FB4FC591D491FB010F
:1024B000E853FB4F649198E014962C91149730E008
:1024C000F901E853FB4F7491F901E452FB4F249159
:1024D000E22FF0E0EE0FFF1FE650FB4F45915491C5
:1024E000FA01208130E0E72FF0E0E095F0952E230F
:1024F0003F23FA01208312962C91129730E0F901C4
:10250000E853FB4F87FF12C05491F901E452FB4F8F
:102510002491E22FF0E0EE0FFF1FE650FB4F2591D4
:102520003491F9014081452B408315C04491F90154
:10253000E452FB4FE491F0E0EE0FFF1FE650FB4F3B
:1025400005911491F801208130E050E040955095BC
:10255000242335232083880F14962C91149730E080
:10256000F901E853FB4F5491F901E452FB4FE49118
:10257000F0E0EE0FFF1FE650FB4F25913491F9017B
:102580004081452B40832881262309F081609150AA
:1025900009F092CF14962C9130E0F901E853FB4FEB
:1025A0009491F901E452FB4F2491E22FF0E0EE0FF9
:1025B000FF1FE650FB4FA591B4912C9130E0E92F1D
:1025C000F0E0E095F0952E233F232C93DF91CF91FF
:1025D0001F910F9108950F931F93CF93DF93DC0109
:1025E000CB0113966C91139770E0FB01E452FB4F03
:1025F000E491F0E0EE0FFF1FE051FB4FC591D49145
:10260000FB01E853FB4F649115962C91159730E030
:10261000F901E853FB4F7491F901E452FB4F249107
:10262000E22FF0E0EE0FFF1FE650FB4F4591549173
:10263000FA01208130E0E72FF0E0E095F0952E23BD
:102640003F23FA01208370E112962C91129730E01B
:10265000F901E853FB4F97FF12C05491F901E4527E
:10266000FB4F2491E22FF0E0EE0FFF1FE650FB4FEF
:1026700025913491F9014081452B408318C0149174
:10268000F901E452FB4F2491E22FF0E0EE0FFF1F1F
:10269000E650FB4F45915491FA01208130E0E12F43
:1026A000F0E0E095F0952E233F23FA012083880F78
:1026B000991F2881262309F0816014962C91149784
:1026C00030E0F901E853FB4F5491F901E452FB4F1C
:1026D000E491F0E0EE0FFF1FE650FB4F259134919F
:1026E000F9014081452B40830000000014962C9195
:1026F000149730E0F901E853FB4F4491F901E4529B
:10270000FB4FE491F0E0EE0FFF1FE650FB4F059109
:102710001491F801208130E050E040955095242339
:1027200035232083715009F08FCF15962C9130E01E
:10273000F901E853FB4F4491F901E452FB4FE49156
:10274000F0E0EE0FFF1FE650FB4FA591B4912C91E6
:10275000242B2C93DF91CF911F910F9108951F93FC
:10276000CF93DF93EC01162F60E08D810E94E8216A
:10277000612F6F77CE010E94421260E0CE010E946D
:102780004212182F61E08D810E94E821812FDF9194
:10279000CF911F910895FC012081318122303105B4
:1027A00019F460E00C94AF1360E070EB0E94EB1240
:1027B00008950F931F93CF93DF93EC018881998144
:1027C0000297A9F468E2CE010E94AF1382FF48C0CD
:1027D00000E010E0CE010E94CB13FE01E00FF11FDC
:1027E000868B0F5F1F4F00341105A1F737C060E0E3
:1027F0008D810E94E821000000008B810E941E2232
:102800008C0161E08D810E94E821012B89F01889FB
:1028100081E0810F888BCE010E94CB13FE01E10F76
:10282000F11D868B0E94F420698B7A8B8B8B9C8B9D
:102830008889811104C08889803280F411C00E9487
:10284000F42009891A892B893C890E5C1F4F2F4F70
:102850003F4F061717072807390768F781E08D8B68
:10286000DF91CF911F910F910895EF92FF921F93E7
:10287000CF93DF931F92CDB7DEB77C01162F60E0B8
:10288000FC01858149830E94E821612F6068C701AE
:102890000E9442124981642FC7010E94421261E0E6
:1028A000F70185810F90DF91CF911F91FF90EF90FD
:1028B0000C94E821CF92DF92EF92FF92CF93DF93B7
:1028C000EC019A01AB01288739874A875B878881A9
:1028D00099810297F1F4CA01B90196958795779588
:1028E0006795785B87419E4F0E948D2A69017A0126
:1028F000432F552763E0CE010E9435144C2D64E030
:10290000CE01DF91CF91FF90EF90DF90CF900C94AC
:102910003514CA01B9010E9400299B01AC0160E88D
:102920007FE588EA98E40E9467286B017C0120E03B
:1029300030E0A9010E940E2A20E030E040E05FE391
:1029400087FD05C0C701B6010E94FF2704C0C7016B
:10295000B6010E94FE270E94CF28615070E0766C7D
:10296000CE01DF91CF91FF90EF90DF90CF900C944C
:10297000EB12CF92DF92EF92FF92CF93DF93EC01B5
:102980004C875D876E877F87888199810297B1F533
:10299000A8EEB3E09A01AB010E94C42AA2E0660F40
:1029A000771F881F991FAA95D1F729E03DE340E0E2
:1029B00050E00E948D2A69017A01B6E0CC0CDD1C42
:1029C000EE1CFF1CBA95D1F7A7016627772767E0B1
:1029D000CE010E94351477276F2D5E2D4D2D68E0B6
:1029E000CE010E9435144C2D69E0CE01DF91CF91CC
:1029F000FF90EF90DF90CF900C943514CB01BA018B
:102A000060567F418D40910925E030E040E050E084
:102A10000E948D2AB9017056CE01DF91CF91FF90AF
:102A2000EF90DF90CF900C94EB12CF93DF93EC01FB
:102A300088819981662369F0029741F461E0CE01B3
:102A40000E94AF13482F437E4C600CC068E372E8CD
:102A500011C0029769F461E0CE010E94AF13482FC4
:102A6000437E446061E0CE01DF91CF910C94351438
:102A700068E072E8CE01DF91CF910C94EB121F93C6
:102A8000CF93DF93EC0188819981029731F440E183
:102A900068E2CE010E94351408C010E460E070EBDB
:102AA000CE010E94EB121150C9F7DF91CF911F9117
:102AB0000895CF93DF93EC01888199816623B9F063
:102AC000029741F461E0CE010E94AF13482F437E8C
:102AD000406116C068EC72E8CE010E94EB1261E81A
:102AE0007AECCE010E94EB1263E87AEC10C00297F8
:102AF00061F461E0CE010E94AF13482F437E446031
:102B000061E0CE010E94351405C068E072E8CE0194
:102B10000E94EB12CE01DF91CF910C943F15CF9321
:102B2000DF93EC01FB01808191818130910529F0D7
:102B3000029731F46AE173E005C063E173E002C01B
:102B400062E273E0CE010E941227CE01DF91CF91A5
:102B500008950F931F93CF93DF9300D000D000D040
:102B6000CDB7DEB78C01FC0187818823B1F067E225
:102B700073E08BE694E00E948D24B801CE010196AB
:102B80000E948F15BE016F5F7F4F8BE694E00E941D
:102B9000AA24CE0101960E94A42661E0F801858155
:102BA0000E94E82160E0C8010E945915F801808167
:102BB0009181029709F056C044E061E0C8010E948B
:102BC000351440E062E0C8010E94351445E065E03C
:102BD000C8010E94351443EC66E0C8010E94351418
:102BE0004FE961E1C8010E9435144FE063E1C8017B
:102BF0000E94351442E469E1C8010E94351440E1A5
:102C000068E2C8010E9435144CED69E2C8010E94D7
:102C1000351448E86EE2C8010E9435144DE26FE2B7
:102C2000C8010E94351444ED60E3C8010E943514C8
:102C300048E067E3C8010E94351440E468E3C80136
:102C40000E9435144FE86CE3C8010E94351442E13C
:102C50006DE3C8010E94351440E36FE6C8010E948D
:102C600035143CC068E072E8C8010E94EB1268EEBF
:102C700070E8C8010E94EB126AE672ECC8010E947B
:102C8000EB1262E17AECC8010E94EB1264ED7EEC7B
:102C9000C8010E94EB1261E874ECC8010E94EB12BB
:102CA00060EA74E9C8010E94EB1267E77CECC80196
:102CB0000E94EB1260E578E9C8010E94EB1260E027
:102CC00070EEC8010E94EB1260E078ECC8010E942F
:102CD000EB1260E470ECC8010E94EB12F80144852D
:102CE000558566857785C8010E94B914F80140852D
:102CF000518562857385C8010E945A14C8010E94DB
:102D00003F1526960FB6F894DEBF0FBECDBFDF91FC
:102D1000CF911F910F910895EF920F93CF93DF936F
:102D2000EC01862F6A834B832C830D83EE821F82F6
:102D300049E553E460E070E0488759876A877B87FC
:102D40004CEC5FE36DE070E04C875D876E877F87BA
:102D5000188A198A1A8A1B8A1C8A1D8A61E00E94B5
:102D6000AF2160E08B810E94AF2161E08C810E94E5
:102D7000AF2161E08D810E94AF2160E08E810E94D1
:102D8000AF2161E08D810E94E82181E090E099838C
:102D900088834AE068E3CE010E94351468E3CE01DF
:102DA0000E94AF138A3079F440E468E3CE010E94B8
:102DB000351468E3CE010E94AF13803421F482E021
:102DC00090E099838883DF91CF910F91EF900895E0
:102DD000FC0167830895FC01608571858285938578
:102DE0000895FC01648575858685978508951F93F0
:102DF000CF93DF93EC01162F60E070E0CE010E94CC
:102E0000EB1297FFF9CF612F70E0786BCE01DF9165
:102E1000CF911F910C94EB128F929F92AF92BF9221
:102E2000DF92EF92FF920F931F93CF93DF93EC010A
:102E30007B01D42E88819981029709F046C06DE309
:102E4000CE010E94AF13482F44606DE3CE010E9473
:102E5000351460E0CE010E945915CE010E943F1545
:102E6000F89460E08D810E94E82160E8CE010E9424
:102E70004212BE2C8701802F8B198D1538F4F80172
:102E800061918F01CE010E944212F5CF61E08D81E8
:102E90000E94E821789461E0CE010E9415150E94FD
:102EA000F4204B015C0168E2CE010E94AF1383FD68
:102EB0003AC00E94F420681979098A099B09643F85
:102EC00071408105910578F5EECF61E0CE010E9459
:102ED00015156AEACE010E94F7166AEACE010E9431
:102EE000F7166AEACE010E94F7166DE2CE010E9443
:102EF000F71664EDCE010E94F7168701AD2CB12CB8
:102F0000C8018E199F098A159B053CF4F80161914F
:102F10008F01CE010E94F716F3CF61E070E080E0F0
:102F200090E00E94232160E0CE010E9415158F8160
:102F3000882361F162E373E08BE694E00E948D24C4
:102F4000E7010D2D10E0CE018E199F098017910722
:102F500074F469914AE050E08BE694E00E94982571
:102F600062E571E08BE694E00E948D24ECCF8BE665
:102F700094E0DF91CF911F910F91FF90EF90DF9040
:102F8000BF90AF909F908F900C949624DF91CF913B
:102F90001F910F91FF90EF90DF90BF90AF909F90A7
:102FA0008F900895FC0140E070E0A1E39F01281B91
:102FB000390B261737076CF4519128E030E0B52F14
:102FC000B427440FB7FD4A27550F21503109B9F7EF
:102FD000EDCF842F089580935D040895EF92FF92C2
:102FE0000F931F93CF93DF931F92CDB7DEB77C0172
:102FF000162F072F63E571E049830E94122749814C
:10300000411102C01FEF0FEF60E2C7010E948B2742
:10301000602FC7010E949E2760E2C7010E948B2794
:10302000612FC7010E949E27C7010F90DF91CF91AA
:103030001F910F91FF90EF900895EF92FF921F93D1
:10304000CF93DF931F92CDB7DEB77C01162F63E5D8
:1030500071E049830E94122760E2C7010E948B271A
:103060004981442319F0612F70E002C06FEF70E0D6
:10307000C7010E94CB27C7010F90DF91CF911F910D
:10308000FF90EF9008959F92AF92BF92CF92DF9200
:10309000EF92FF920F931F93CF93DF9300D000D056
:1030A00000D0CDB7DEB75C018B0163E571E00E9413
:1030B0001227F801948081E0982687818823C9F03F
:1030C000C584D684E784F08820E030E040E252EC0A
:1030D000C701B6010E94632887FD0AC02AE939E9C1
:1030E0004FE652E4C701B6010E940E2A18160CF4EE
:1030F000912CF8018085882329F0818981508336BD
:1031000008F0CCC0992009F4C9C061E473E0C5019E
:103110000E947B27F8016181C5010E949E2768E417
:1031200073E0C5010E947B2720E030E040E251E4DB
:10313000F80165857685878590890E94122A20E0AE
:1031400030E04AE754E40E94FF270E94D428F801A7
:103150004781CE0101960E94EE17BE016F5F7F4F3F
:10316000C5010E947427CE0101960E94A426F80191
:1031700040856189CE0101960E941D18BE016F5FD6
:103180007F4FC5010E947427CE0101960E94A4269C
:10319000F80162897389848995890E94D428F8018D
:1031A0004185CE0101960E94EE17BE016F5F7F4FF1
:1031B000C5010E947427CE0101960E94A42620E03A
:1031C00030E040E251E4F80166897789808D918D85
:1031D0000E94122A0E94D428F8014385CE0101964C
:1031E0000E94EE17BE016F5F7F4FC5010E947427DA
:1031F000CE0101960E94A42620E030E040E251E496
:10320000F801628D738D848D958D0E94122A0E9423
:10321000D428F8014285CE0101960E94EE17BE0126
:103220006F5F7F4FC5010E947427CE0101960E94F7
:10323000A42620E030E040E251E4F801668D778D6D
:1032400080A191A10E94122A0E94D428F8014485ED
:10325000CE0101960E94EE17BE016F5F7F4FC50140
:103260000E947427CE0101960E94A426F801628173
:10327000848181116E5FF801838181116C5F41E06F
:10328000CE0101960E941D18BE016F5F7F4FC501E0
:103290000E947427CE0101960E94A426C50126969D
:1032A0000FB6F894DEBF0FBECDBFDF91CF911F9157
:1032B0000F91FF90EF90DF90CF90BF90AF909F90D5
:1032C0000895FC0181818F70880F8D5F08952F9282
:1032D0003F924F925F926F927F928F929F92AF92A6
:1032E000BF92CF92DF92EF92FF920F931F93CF93F3
:1032F000DF93CDB7DEB763970FB6F894DEBF0FBE8E
:10330000CDBF8C010E9461198150FE0139969E014A
:103310002F5E3F4F1192E217F307E1F72889AF8440
:10332000CE848D849C84DB84EA84B984D801682FA0
:1033300070E091E0AD01401B510B461757070CF0B0
:1033400078C08D91AE014F5F5F4FF22E20E030E0EC
:10335000E82FE170E98BF82FF270FB8BE82FE47017
:103360006E2EF82FF8705F2EE82FE0714E2EF82F9A
:10337000F0723F2EE82FE0742E2EF9013197E730DE
:10338000F10520F4E25BFF4F0C94AF2AE82FEE0F1B
:10339000EE0BE923E9832BC0222011F09A8327C08A
:1033A0001A8225C0332011F09B8321C01B821FC0CD
:1033B000442011F09C831BC01C8219C0552011F0C1
:1033C0009D8315C01D8213C0662011F09E830FC01F
:1033D0001E820DC0FB89FF2311F09F8308C01F824E
:1033E00006C07988772011F0988701C01886FA0105
:1033F0007190AF017A8AE72DE13009F4F724F82DB6
:10340000FF25892C8F242F5F3F4F2830310549F04D
:10341000EA2DAC2CCF2E9D2CDE2CEB2CBF2CFE2EBF
:10342000ACCF2A2DAC2CCF2E9D2CDE2CEB2CBF2C20
:1034300081CFF0E82F9F9001112440E4A49EC001A9
:103440001124822B8B2990E2C99E90011124822B9A
:10345000E0E18E9E90011124822BF8E09F9E900166
:103460001124822B44E0D49E90011124822BEE0C77
:103470008E2963960FB6F894DEBF0FBECDBFDF91E5
:10348000CF911F910F91FF90EF90DF90CF90BF9061
:10349000AF909F908F907F906F905F904F903F90F4
:1034A0002F900895CF92DF92EF92FF92CF93DF9308
:1034B000D62FC42F24E6829FC0011124BC01882787
:1034C00077FD8095982F0E94022920E030E0A90125
:1034D0000E94FF276B017C018AE0D89FB001112474
:1034E000882777FD8095982F0E9402299B01AC01C7
:1034F000C701B6010E94FF276B017C016C2F70E0B1
:1035000080E090E00E9402299B01AC01C701B60156
:103510000E94FF27DF91CF91FF90EF90DF90CF9037
:1035200008957F928F929F92AF92BF92CF92DF9237
:10353000EF92FF920F931F93CF93DF938C01EB01D8
:1035400081E08E83188219821A821B821C821F825C
:10355000188619861A861B861C861D861E861F865F
:10356000188A198A1A8A1B8A1C8A1D8A1E8A1F8A2F
:10357000188E198E1A8E1B8E1C8E1D8E1E8E1F8EFF
:1035800018A219A21D82C8010E946119F801E80F52
:10359000F11D3197F080FD82C8010E946719F81271
:1035A0001E82F801808182958F7088838A3009F0AD
:1035B0001E828E81882309F4E0C0F80180818F701B
:1035C000F4E08F9FC0011124F801918192959695A6
:1035D00096959370982B9983918181E095FF80E077
:1035E0008A83F801918181E094FF80E08C83F80167
:1035F00081818F700D5F1F4FE12CF12CC82ED12CD3
:1036000077247394EC14FD040CF0B7C0FFEFEF1AAD
:10361000FF0AF80131979081F8016081892F8F703E
:10362000B62EB2942FE0B2226F70A62E92959F70A4
:10363000923009F45CC030F4992311F1913009F40F
:1036400049C098C0933009F46CC0943009F092C01E
:103650007C8670E080E1B89E600D711D1124882782
:1036600077FD8095982F0E94022920E030E040E20B
:1036700051E40E9467286E8F7F8F88A399A37AC038
:103680007F82462F6B2D0E94521A20E030E048ECDA
:1036900053E40E94FE2720E030E040E251E40E9423
:1036A00067284B015C016D877E878F87988B20E0B0
:1036B00030E040E752E40E940E2A1816B4F020E0F1
:1036C00030E040E252ECC501B4010E94632887FF5C
:1036D00051C00BC09887462F6B2D0E94521A0E9432
:1036E000D428698B653608F445C01E8243C07986AC
:1036F0006B2D70E0F0E18F9F600D711D112484E04F
:10370000660F771F8A95E1F76A0D711D882777FD8F
:103710008095982F0E9402296A8B7B8B8C8B9D8BC6
:1037200029C07B867A86682F70E080E090E00E9456
:10373000022920E030E044EB51E40E94122A6E8B13
:103740007F8B888F998F6A2D70E020E1B29E600D8B
:10375000711D1124882777FD8095982F0E940229DA
:1037600020E030E040E251E40E9467286A8F7B8FBE
:103770008C8F9D8F0E5F1F4F45CFDF91CF911F9193
:103780000F91FF90EF90DF90CF90BF90AF909F9000
:103790008F907F900895CF92DF92EF92FF920F93D8
:1037A0001F93CF93DF93CDB7DEB7A2970FB6F894F0
:1037B000DEBF0FBECDBF8C01BE016F5F7F4F0E9489
:1037C000911AC8010E946119C82E8F81882321F1A6
:1037D0006BE473E08BE694E00E948D247801D12C99
:1037E000C701801B910B8C159D0584F4F701619135
:1037F0007F0140E150E08BE694E00E94982562E56D
:1038000071E08BE694E00E948D24EACF66E072E0DE
:103810008BE694E00E948D248F81882309F4F8C000
:1038200063E172E08BE694E00E948D246BE172E02C
:103830008BE694E00E948D2440E150E069818BE6A4
:1038400094E00E9498256FE172E08BE694E00E947C
:103850008D2440E150E06A818BE694E00E94982537
:103860006DE572E08BE694E00E948D246B8170E040
:103870004AE050E08BE694E00E94832564E573E023
:103880008BE694E00E948D246C8170E04AE050E069
:103890008BE694E00E9483256EE573E08BE694E06E
:1038A0000E948D246D8170E04AE050E08BE694E048
:1038B0000E9483256FE672E08BE694E00E948D24DF
:1038C0008885882359F04E855F856889798922E04B
:1038D00030E08BE694E00E94902606C066E673E036
:1038E0008BE694E00E948D2461E872E08BE694E020
:1038F0000E948D248985882341F04AE050E06A893E
:103900008BE694E00E94982506C066E673E08BE69D
:1039100094E00E948D246AE673E08BE694E00E94B6
:103920008D248A85882359F04B895C896D897E892D
:1039300022E030E08BE694E00E94902606C066E626
:1039400073E08BE694E00E948D2461E773E08BE6E0
:1039500094E00E948D248B85882369F04B8D5C8DCB
:103960006D8D7E8D22E030E08BE694E00E94902603
:1039700067E873E002C066E673E08BE694E00E94BD
:103980008D2468E773E08BE694E00E948D248C859B
:10399000882359F04F89588D698D7A8D22E030E067
:1039A0008BE694E00E94902606C066E673E08BE604
:1039B00094E00E948D246FE773E08BE694E00E9410
:1039C0008D248D85882369F04F8D58A169A17AA136
:1039D00022E030E08BE694E00E94902666E873E0F7
:1039E00002C066E673E08BE694E00E948D2465E4F5
:1039F00072E08BE694E00E948D2440E150E06E81FD
:103A00008BE694E00E9498258BE694E00E94962431
:103A1000A2960FB6F894DEBF0FBECDBFDF91CF9157
:103A20001F910F91FF90EF90DF90CF9008950F932B
:103A30001F93CF93DF93CDB7DEB7AE970FB6F89451
:103A4000DEBF0FBECDBF8C0163E571E0CE0189966C
:103A50000E941227F8018081807A803A31F5BE01F8
:103A60006F5F7F4FC8010E94911A8F81882391F068
:103A7000BE016F5F7F4FCE0183960E944318BE0147
:103A80006D5D7F4FCE0189960E942827CE018396D7
:103A90000E94A4268DA59EA5892B39F0BE01675DE5
:103AA0007F4F8BE694E00E94AA2411E02DA53EA54D
:103AB000232B09F410E0CE0189960E94A426812FC1
:103AC000AE960FB6F894DEBF0FBECDBFDF91CF919B
:103AD0001F910F910895FC0120E030E080E0A1E308
:103AE000919140E050E0BA01620F731F643171059B
:103AF00034F4692F6827880F67FD8A27990F4F5F75
:103B00005F4F4830510579F7285F3F4F2831310525
:103B100039F70895FF920F931F93CF93DF938C0192
:103B2000EB0181E08B87F8018281F0E18F9FC0017A
:103B30001124F801F380F294AFE0FA22F82AF98612
:103B4000C8010E946B1DF8121B86F80180818F73DB
:103B5000898380818295869586958370888383305A
:103B600009F01B86F8019181892F881F8827881FFB
:103B70008A83818186FB882780F98B8361816F73BB
:103B8000F0E16F9FB0011124F801828182958F705E
:103B9000682B882777FD8095982F0E9402292DECAD
:103BA0003CEC4CEC5DE30E94122A20E030E040E265
:103BB00052E40E94FE276C837D838E839F83F801ED
:103BC00083818F708A878AE68887DF91CF911F91E2
:103BD0000F91FF900895AF92BF92CF92DF92EF9234
:103BE000FF920F931F93CF93DF9300D000D000D0AC
:103BF000CDB7DEB75C018B0163E571E0CE010196C4
:103C00000E94122767E572E0CE0101960E947B2791
:103C1000F8016181CE0101960E949E2760E2CE01EB
:103C200001960E948B27F80180858F77843610F0EB
:103C30008A3651F4F8018281882319F061E870E036
:103C400008C061E070E005C08D3709F042C062E84D
:103C500070E0CE0101960E94CB2760E2CE01019672
:103C60000E948B2720E030E040E251E4F8016481BB
:103C70007581868197810E94122A20E030E04AE710
:103C800054E40E94FF270E94D428F62E672FCE010D
:103C900001960E949E2760E2CE0101960E948B272A
:103CA0006F2DCE0101960E949E2760E2CE01019603
:103CB0000E948B27F801C480D580E680F78020E041
:103CC00030E040E752E4C701B6010E940E2A87FDAA
:103CD00006C063E571E0C5010E94122719C020E00B
:103CE00030E040E252ECC701B6010E94632818168A
:103CF00084F7F8016085838181116068CE010196A7
:103D00000E949E27BE016F5F7F4FC5010E943F2723
:103D1000CE0101960E94A426C50126960FB6F894FE
:103D2000DEBF0FBECDBFDF91CF911F910F91FF90EE
:103D3000EF90DF90CF90BF90AF900895EF92FF92F9
:103D40000F931F93CF93DF93CDB7DEB7A1970FB635
:103D5000F894DEBF0FBECDBF7C01BE016F5E7F4F0A
:103D60000E948A1D1D8E1E8E1F8E18A219A22A89DE
:103D7000FE017D96CE0182963191231709F4C0C0D1
:103D8000E817F907C9F70E94F42000915E0410912A
:103D90005F042091600430916104601B710B820B01
:103DA000930B9F938F937F936F9386EF91E09F93F5
:103DB0008F938E010F5F1F4F1F930F930E94142D3F
:103DC0000E94F42060935E0470935F04809360040B
:103DD00090936104B8018BE694E00E948D246BE817
:103DE00073E08BE694E00E948D2487010FB6F8946F
:103DF000DEBF0FBECDBFE12CF12CF80161918F0128
:103E00004AE050E08BE694E00E94982562E571E07C
:103E10008BE694E00E948D24FFEFEF1AFF0A84E006
:103E2000E816F10451F766E072E08BE694E00E9438
:103E30008D248C8D811107C068E072E08BE694E0E0
:103E40000E948D2459C063E172E08BE694E00E94E9
:103E50008D246BE172E08BE694E00E948D244AE0B1
:103E600050E069898BE694E00E9498256FE172E04A
:103E70008BE694E00E948D244AE050E06A898BE64C
:103E800094E00E9498256DE572E08BE694E00E9434
:103E90008D246B8970E04AE050E08BE694E00E944C
:103EA000832566E772E08BE694E00E948D246C899E
:103EB00070E04AE050E08BE694E00E9483256FE6D4
:103EC00072E08BE694E00E948D244D895E896F89B3
:103ED000788D22E030E08BE694E00E94902665E445
:103EE00072E08BE694E00E948D244AE050E06A8DF7
:103EF0008BE694E00E9498258BE694E00E9496243D
:103F0000A1960FB6F894DEBF0FBECDBFDF91CF9163
:103F10001F910F91FF90EF9008950F931F93CF93F0
:103F2000DF93CDB7DEB768970FB6F894DEBF0FBE4C
:103F3000CDBF8C0163E571E0CE0143960E9412274C
:103F4000F8018081807C803C31F5BE016F5F7F4F3E
:103F5000C8010E948A1D8C85882391F0BE016F5F85
:103F60007F4FCE010D960E94EB1DBE01635F7F4F18
:103F7000CE0143960E942827CE010D960E94A426CA
:103F80008F89988D892B39F0BE016D5E7F4F8BE64E
:103F900094E00E94AA2411E02F89388D232B09F484
:103FA00010E0CE0143960E94A426812F68960FB69A
:103FB000F894DEBF0FBECDBFDF91CF911F910F915F
:103FC000089520E030E040E0FC015191CF01450F21
:103FD0002F5F3F4F26303105B9F781E0411180E076
:103FE0000895CF92DF92EF92FF920F931F93CF939A
:103FF000DF938C01EB0181E08B87F801808188835E
:1040000085818A87C8010E94E11F8B87F801918111
:10401000292F2F70907392959F7009F494E0F0E12E
:104020009F9FC0011124822B8983F801628170E077
:1040300062537109882777FD8095982F0E94022985
:1040400020E030E040E251E40E94122A6B017C0142
:10405000F801638170E080E090E00E9402299B01FA
:10406000AC01C701B6010E94FF2720E030E040E22A
:1040700051E40E9467286C837D838E839F83F801BF
:1040800084818987818190E026E0959587952A959E
:10409000E1F721E0892B09F420E02887DF91CF9117
:1040A0001F910F91FF90EF90DF90CF9008950F93A5
:1040B0001F93CF93DF93CDB7DEB768970FB6F89411
:1040C000DEBF0FBECDBF8C0163E571E0CE0143962C
:1040D0000E941227F8018081813531F5BE016F5FA2
:1040E0007F4FC8010E94F11F8C85882391F0BE018B
:1040F0006F5F7F4FCE010D960E94E10CBE01635FA2
:104100007F4FCE0143960E942827CE010D960E9434
:10411000A4268F89988D892B39F0BE016D5E7F4F63
:104120008BE694E00E94AA2411E02F89388D232B7E
:1041300009F410E0CE0143960E94A426812F6896D0
:104140000FB6F894DEBF0FBECDBFDF91CF911F91A8
:104150000F9108951F920F920FB60F9211242F9373
:104160003F938F939F93AF93BF93809163049091FC
:104170006404A0916504B09166043091620423E068
:10418000230F2D3720F40196A11DB11D05C026E88F
:10419000230F0296A11DB11D209362048093630436
:1041A00090936404A0936504B093660480916704BF
:1041B00090916804A0916904B0916A040196A11DD0
:1041C000B11D8093670490936804A0936904B09331
:1041D0006A04BF91AF919F918F913F912F910F9062
:1041E0000FBE0F901F9018952FB7F894609163043D
:1041F0007091640480916504909166042FBF0895C6
:104200003FB7F8948091670490916804A091690485
:10421000B0916A0426B5A89B05C02F3F19F00196FE
:10422000A11DB11D3FBF6627782F892F9A2F620FDE
:10423000711D811D911D42E0660F771F881F991F18
:104240004A95D1F70895CF92DF92EF92FF92CF93E4
:10425000DF936B017C010E940021EB01C114D104AA
:10426000E104F10489F00E94FD270E9400216C1BEB
:104270007D0B683E734090F381E0C81AD108E108D5
:10428000F108C851DC4FEACFDF91CF91FF90EF905A
:10429000DF90CF900895789484B5826084BD84B512
:1042A000816084BD85B5826085BD85B5816085BD31
:1042B000EEE6F0E0808181608083E1E8F0E010824A
:1042C000808182608083808181608083E0E8F0E08B
:1042D000808181608083E1EBF0E080818460808375
:1042E000E0EBF0E0808181608083EAE7F0E08081AC
:1042F000846080838081826080838081816080830C
:104300008081806880831092C1000895833081F09D
:1043100028F4813099F08230A1F008958730A9F017
:104320008830B9F08430D1F4809180008F7D03C053
:10433000809180008F7780938000089584B58F7777
:1043400002C084B58F7D84BD08958091B0008F77C1
:1043500003C08091B0008F7D8093B0000895CF930B
:10436000DF9390E0FC01E853FB4F2491FC01E45201
:10437000FB4F8491882349F190E0880F991FFC013D
:10438000EC5FFA4FA591B49186509B4FFC01C5910B
:10439000D4919FB7611108C0F8948C912095822325
:1043A0008C93888182230AC0623051F4F8948C91F6
:1043B000322F309583238C938881822B888304C08D
:1043C000F8948C91822B8C939FBFDF91CF910895AD
:1043D0000F931F93CF93DF931F92CDB7DEB7282F94
:1043E00030E0F901EC54FB4F8491F901E853FB4FA5
:1043F0001491F901E452FB4F04910023C9F0882382
:1044000021F069830E9486216981E02FF0E0EE0FA0
:10441000FF1FE650FB4FA591B4919FB7F8948C9184
:10442000611103C01095812301C0812B8C939FBF24
:104430000F90DF91CF911F910F910895CF93DF934C
:10444000282F30E0F901EC54FB4F8491F901E85337
:10445000FB4FD491F901E452FB4FC491CC2391F06E
:1044600081110E948621EC2FF0E0EE0FFF1FE0513A
:10447000FB4FA591B4912C912D2381E090E021F484
:1044800080E002C080E090E0DF91CF910895FC01D0
:10449000818D228D90E0805C9F4F821B91098F73EC
:1044A00099270895FC01918D828D981731F0828DA6
:1044B000E80FF11D858D90E008958FEF9FEF08952F
:1044C000FC01918D828D981761F0828DDF01A80F1C
:1044D000B11D5D968C91928D9F5F9F73928F90E03E
:1044E00008958FEF9FEF089584EE93E2892B49F0B2
:1044F00080E090E0892B29F00E94E42381110C9444
:1045000000000895FC01848DDF01A80FB11DA35A9E
:10451000BF4F2C91848D90E001968F739927848FE3
:10452000A689B7892C93A089B1898C9180648C93DA
:10453000938D848D981306C00288F389E02D8081C5
:104540008F7D80830895CF93DF93EC01888D88233E
:10455000C9F0EA89FB89808185FD05C0A889B989F0
:104560008C9186FD0FC00FB607FCF5CF808185FFCB
:10457000F2CFA889B9898C9185FFEDCFCE010E9439
:104580008222E7CFDF91CF910895CF92DF92FF9201
:104590000F931F93CF93DF931F92CDB7DEB76C01BC
:1045A000DC015B969C915B975C968C915C97981371
:1045B00007C05096ED91FC915197808185FD32C0E6
:1045C000F601038D10E00F5F1F4F0F731127F02EC0
:1045D000F601848DF81211C00FB607FCF9CFD60191
:1045E0005096ED91FC915197808185FFF1CFC601E6
:1045F00069830E9482226981EBCF838DE80FF11DD0
:10460000E35AFF4F6083D6015B960C935B975296FB
:10461000ED91FC91539780818062808381E0589670
:104620008C930DC0D6015696ED91FC9157976083FF
:104630005096ED91FC91519780818064808381E058
:1046400090E00F90DF91CF911F910F91FF90DF903D
:10465000CF900895BF92CF92DF92EF92FF92CF93C7
:10466000DF93EC016A017B01B22EE889F98982E0CF
:104670008083411581EE580761057105A1F060E066
:1046800079E08DE390E0A70196010E948D2A2150E8
:1046900031094109510956954795379527952115B7
:1046A00080E1380798F0E889F989108260E874E8B9
:1046B0008EE190E0A70196010E948D2A21503109D8
:1046C000410951095695479537952795EC85FD8504
:1046D0003083EE85FF852083188EEC89FD89B082BA
:1046E000EA89FB89808180618083EA89FB898081F6
:1046F00088608083EA89FB89808180688083EA8979
:10470000FB8980818F7D8083DF91CF91FF90EF9037
:10471000DF90CF90BF9008951F920F920FB60F9227
:1047200011242F938F939F93EF93FF93E0917B043A
:10473000F0917C048081E0918104F091820482FDFB
:1047400012C09081809184048F5F8F7320918504C3
:10475000821751F0E0918404F0E0E559FB4F958F0A
:104760008093840401C08081FF91EF919F918F918C
:104770002F910F900FBE0F901F9018951F920F92C0
:104780000FB60F9211242F933F934F935F936F9324
:104790007F938F939F93AF93BF93EF93FF938BE69A
:1047A00094E00E948222FF91EF91BF91AF919F917F
:1047B0008F917F916F915F914F913F912F910F90CA
:1047C0000FBE0F901F9018958BE694E00E94472231
:1047D00021E0892B09F420E0822F089510926E04C5
:1047E00010926D0488EE93E0A0E0B0E080936F0437
:1047F00090937004A0937104B093720488E993E0DD
:1048000090936C0480936B0485EC90E09093780413
:104810008093770484EC90E090937A0480937904F9
:1048200080EC90E090937C0480937B0481EC90E09A
:1048300090937E0480937D0482EC90E090938004BA
:1048400080937F0486EC90E09093820480938104AF
:1048500010928404109285041092860410928704AA
:10486000089508950E944B210E9431240E943D0426
:10487000C4E7D2E20E94B5042097E1F30E947422BB
:10488000F9CFCF92DF92EF92FF920F931F93CF93C6
:10489000DF936C017A01EB01E60EF71E00E010E0F9
:1048A000CE15DF0561F06991D601ED91FC91019083
:1048B000F081E02DC6010995080F191FF1CFC8013D
:1048C000DF91CF911F910F91FF90EF90DF90CF90EC
:1048D00008956115710581F0DB010D900020E9F765
:1048E000AD0141505109461B570BDC01ED91FC9184
:1048F0000280F381E02D099480E090E00895DC01CE
:10490000ED91FC91DB0114964D915C9115976D91A1
:104910007C910280F381E02D09940C946924DC01E0
:10492000ED91FC910190F081E02D09940F931F937C
:10493000CF93DF93EC016DE00E948F248C016AE03D
:10494000CE010E948F24800F911FDF91CF911F9184
:104950000F9108950F931F93CF93DF93EC010E9463
:104960007F248C01CE010E949624800F911FDF913D
:10497000CF911F910F9108950F931F93CF93DF93C2
:10498000EC010E9469248C01CE010E949624800FC4
:10499000911FDF91CF911F910F9108950F931F9356
:1049A000CF93DF93EC010E948F248C01CE010E94F3
:1049B0009624800F911FDF91CF911F910F91089541
:1049C0008F929F92AF92BF92CF92DF92EF92FF921F
:1049D0000F931F93CF93DF93CDB7DEB7A1970FB699
:1049E000F894DEBF0FBECDBF7C01C42EE52FCB01F6
:1049F000D22E19A221E02D1510F02AE0D22E8E0120
:104A00000F5D1F4F8D2C912CA12CB12C6C2D7E2F66
:104A1000A50194010E948D2A8C2DD29E801911240B
:104A2000015011098A3014F4805D01C0895CF801DD
:104A30008083211531054105510521F0C22EE32F58
:104A4000CA01E4CFB801C7010E946924A1960FB63C
:104A5000F894DEBF0FBECDBFDF91CF911F910F91B4
:104A6000FF90EF90DF90CF90BF90AF909F908F908E
:104A70000895CF92DF92EF92FF920F931F93CF93FF
:104A8000DF93EC016A017B012115310579F4E8819E
:104A9000F9810190F081E02D642FDF91CF911F917A
:104AA0000F91FF90EF90DF90CF9009942A3031055D
:104AB000E9F477FF1AC06DE20E948F248C0144272D
:104AC0005527BA014C195D096E097F092AE0CE010C
:104AD0000E94E024800F911FDF91CF911F910F91D1
:104AE000FF90EF90DF90CF9008952AE0B701A601E4
:104AF000CE01DF91CF911F910F91FF90EF90DF904A
:104B0000CF900C94E0249A01AB01662757FD609585
:104B1000762F0C9439252115310541F4DC01ED91F6
:104B2000FC910190F081E02D642F09940C94E02415
:104B30009A01462F50E060E070E00C948B259A01BA
:104B4000AB0160E070E00C948B254F925F926F9206
:104B50007F928F929F92AF92BF92CF92DF92EF920D
:104B6000FF920F931F93CF93DF93EC016A017B01B8
:104B7000B22E9A01AB01C701B6010E94752A8823A3
:104B800019F064EA73E027C026013701E89477F84A
:104B90002FEF3FEF4FE75FE7C301B2010E94752A95
:104BA00081110DC02FEF3FEF4FE75FE7C301B20167
:104BB0000E94632818161CF468EA73E00CC02FEFFB
:104BC0003FEF4FE75FE4C701B6010E940E2A1816B7
:104BD000ACF46CEA73E0CE01DF91CF911F910F919D
:104BE000FF90EF90DF90CF90BF90AF909F908F900D
:104BF0007F906F905F904F900C9469242FEF3FEF60
:104C00004FE75FECC701B6010E94632887FDE1CF43
:104C100020E030E0A901C701B6010E94632887FFA8
:104C20000AC06DE2CE010E948F248C01F7FAF09445
:104C3000F7F8F09402C000E010E0A12C60E070E012
:104C400080E09FE3AB1441F020E030E040E251E42B
:104C50000E946728A394F6CF9B01AC01C701B6015F
:104C60000E94FF276B017C010E94D4282B013C018C
:104C70000E9400299B01AC01C701B6010E94FE27DA
:104C80006B017C012AE0B301A201CE010E94E02465
:104C9000080F191FBB2039F060EB73E0CE010E94B2
:104CA0006924080F191F7B2C772041F120E030E0A8
:104CB00040E251E4C701B6010E94122A6B017C0157
:104CC0000E94CF284B01AA2497FCA094BA2C2AE07A
:104CD00030E0B501A401CE010E943925080F191F4B
:104CE000C501B4010E9402299B01AC01C701B601B4
:104CF0000E94FE276B017C017A94D6CFC801DF9118
:104D0000CF911F910F91FF90EF90DF90CF90BF90C8
:104D1000AF909F908F907F906F905F904F9008958D
:104D20000C94A5250F931F93CF93DF93EC010E9462
:104D3000A5258C01CE010E949624800F911FDF9142
:104D4000CF911F910F910895FC01808191810C9466
:104D50007B2BCF93DF93EC0188819981009711F031
:104D60000E947B2B198218821D821C821B821A8250
:104D7000DF91CF9108950F931F93CF93DF93EC01B1
:104D80008B016F5F7F4F888199810E940A2C009769
:104D900031F0998388831B830A8381E001C080E01E
:104DA000DF91CF911F910F910895CF93DF93EC0185
:104DB00088819981892B29F08A819B8186179707A1
:104DC00060F4CE010E94BB26882341F08C819D8136
:104DD000892B19F4E881F981108281E0DF91CF916C
:104DE0000895EF92FF920F931F93CF93DF93EC01FF
:104DF0007B018A01BA010E94D526811104C0CE012F
:104E00000E94A92607C01D830C83B7018881998160
:104E10000E94DD2CCE01DF91CF911F910F91FF9069
:104E2000EF900895FC011182108213821282158284
:104E300014826115710559F0FB0101900020E9F71A
:104E4000AF0141505109461B570B0C94F1260895B0
:104E5000CF93DF93EC01FB018617970761F0608128
:104E600071816115710529F0448155810E94F126F7
:104E700002C00E94A926CE01DF91CF910895FC01C6
:104E80001182108213821282158214820C942827B8
:104E9000EF92FF920F931F93CF93DF93EC017B016F
:104EA0000C811D816115710511F480E016C041155A
:104EB000510591F0040F151FB8010E94D5268823D3
:104EC000A1F3288139818C819D81B701820F931FC5
:104ED0000E94DD2C1D830C8381E0DF91CF911F9117
:104EE0000F91FF90EF900895FB01448155816081FF
:104EF00071810C9448276115710559F0FB010190EF
:104F00000020E9F7AF0141505109461B570B0C94A3
:104F1000482780E00895CF93DF9300D0CDB7DEB768
:104F200069831A8241E050E0BE016F5F7F4F0E94AB
:104F300048270F900F90DF91CF910895EF92FF9245
:104F40000F931F93CF93DF9300D000D0CDB7DEB780
:104F50007C01862F4AE050E08E010F5F1F4FB801A1
:104F600090E00E94E42CF80101900020E9F7AF01E5
:104F700041505109401B510BB801C7010E944827FD
:104F80000F900F900F900F90DF91CF911F910F9185
:104F9000FF90EF900895EF92FF920F931F93CF939E
:104FA000DF93CDB7DEB728970FB6F894DEBF0FBEFC
:104FB000CDBF7C01CB014AE050E08E010F5F1F4F57
:104FC000B8010E94E42CF80101900020E9F7AF013C
:104FD00041505109401B510BB801C7010E9448279D
:104FE00028960FB6F894DEBF0FBECDBFDF91CF91EC
:104FF0001F910F91FF90EF90089508955058BB278F
:10500000AA270ED0D1C1C2D130F0C7D120F031F4DF
:105010009F3F11F41EF4B7C10EF4E095E7FB9FC16A
:10502000E92FD3D180F3BA17620773078407950776
:1050300018F071F49EF5EBC10EF4E0950B2EBA2F2B
:10504000A02D0B01B90190010C01CA01A00111248E
:10505000FF27591B99F0593F50F4503E68F11A163A
:10506000F040A22F232F342F4427585FF3CF4695CB
:1050700037952795A795F0405395C9F77EF41F16ED
:10508000BA0B620B730B840BBAF09150A1F0FF0FB7
:10509000BB1F661F771F881FC2F70EC0BA0F621FA3
:1050A000731F841F48F4879577956795B795F79593
:1050B0009E3F08F0B3CF9395880F08F09927EE0F25
:1050C00097958795089527D108F481E008950CD02D
:1050D0006BC163D140F05AD130F021F45F3F19F039
:1050E0003EC1511195C14FC170D198F39923C9F3B5
:1050F0005523B1F3951B550BBB27AA2762177307DE
:10510000840738F09F5F5F4F220F331F441FAA1F91
:10511000A9F333D00E2E3AF0E0E830D09150504051
:10512000E695001CCAF729D0FE2F27D0660F771FFF
:10513000881FBB1F261737074807AB07B0E809F0E1
:10514000BB0B802DBF01FF2793585F4F2AF09E3F76
:10515000510568F004C15CC15F3FECF3983EDCF39D
:10516000869577956795B795F7959F5FC9F7880FEF
:10517000911D9695879597F90895E1E0660F771F41
:10518000881FBB1F621773078407BA0720F0621BD2
:10519000730B840BBA0BEE1F88F7E095089504D0CB
:1051A0006894B11135C1089518D188F09F5790F0D7
:1051B000B92F9927B751A0F0D1F0660F771F881F3C
:1051C000991F1AF0BA95C9F712C0B13081F01FD1FA
:1051D000B1E008951CC1672F782F8827B85F39F098
:1051E000B93FCCF3869577956795B395D9F73EF49B
:1051F00090958095709561957F4F8F4F9F4F089543
:10520000E89409C097FB3EF4909580957095619560
:105210007F4F8F4F9F4F9923A9F0F92F96E9BB2716
:105220009395F695879577956795B795F111F8CF92
:10523000FAF4BB0F11F460FF1BC06F5F7F4F8F4FFD
:105240009F4F16C0882311F096E911C0772321F0F3
:105250009EE8872F762F05C0662371F096E8862F8B
:1052600070E060E02AF09A95660F771F881FDAF7E2
:10527000880F9695879597F9089588D018F011F0C2
:105280008CD038F480C0C4C0E92F9FD0B0F3552330
:10529000C9F3E7FB6217730784079507A8F199F331
:1052A000E92FFF2788232AF03197660F771F881F81
:1052B000DAF7952F5527442332F091505040220FB2
:1052C000331F441FD2F7BB27E91BF50B621B730B7F
:1052D000840BB109C1F222F4620F731F841FB11D48
:1052E00031972AF0660F771F881FBB1FEFCF9150B1
:1052F00050405AF041F0882332F0660F771F881F24
:1053000091505040C1F7939530C086957795679539
:105310009F5FD9F7F8CF990F0008550FAA0BE0E867
:10532000FEEF16161706E807F907C0F01216130667
:10533000E407F50798F0621B730B840B950B39F4A7
:105340000A2661F0232B242B252B21F408950A260D
:1053500009F4A140A6958FEF811D811D089597F94D
:105360009F6780E870E060E008959F3F31F09150C2
:1053700020F4879577956795B795880F911D969539
:10538000879597F908959FEF80EC089500240A947B
:105390001616170618060906089500240A94121610
:1053A0001306140605060895092E0394000C11F443
:1053B000882352F0BB0F40F4BF2B11F460FF04C0F0
:1053C0006F5F7F4F8F4F9F4F089557FD9058440F49
:1053D000551F59F05F3F71F04795880F97FB991F54
:1053E00061F09F3F79F08795089512161306140611
:1053F000551FF2CF4695F1DF08C01616170618069E
:10540000991FF1CF86957105610508940895E89478
:10541000BB2766277727CB0197F908957CDF08F42F
:105420008FEF08950BD0C0CFB1DF28F0B6DF18F0B2
:10543000952309F094CFA7CF1124EACFC6DFA0F3BC
:10544000959FD1F3950F50E0551F629FF001729F19
:10545000BB27F00DB11D639FAA27F00DB11DAA1F38
:10546000649F6627B00DA11D661F829F2227B00D85
:10547000A11D621F739FB00DA11D621F839FA00D10
:10548000611D221F749F3327A00D611D231F849F60
:10549000600D211D822F762F6A2F11249F575040B7
:1054A0008AF0E1F088234AF0EE0FFF1FBB1F661F52
:1054B000771F881F91505040A9F79E3F510570F00B
:1054C0004ECFA6CF5F3FECF3983EDCF38695779501
:1054D0006795B795F795E7959F5FC1F7FE2B880F06
:1054E000911D9695879597F9089515DF880B990B6F
:1054F000089597FB072E16F4009407D077FD09D086
:105500000E94CF2A07FC05D03EF4909581959F4FCD
:105510000895709561957F4F0895A1E21A2EAA1BF8
:10552000BB1BFD010DC0AA1FBB1FEE1FFF1FA21753
:10553000B307E407F50720F0A21BB30BE40BF50B50
:10554000661F771F881F991F1A9469F760957095D9
:10555000809590959B01AC01BD01CF010895EE0FA0
:10556000FF1F0590F491E02D0994A29FB001B39F15
:10557000C001A39F700D811D1124911DB29F700D5C
:10558000811D1124911D08950E94B52AA59F900D9B
:10559000B49F900DA49F800D911D11240895AA1B06
:1055A000BB1B51E107C0AA1FBB1FA617B70710F00E
:1055B000A61BB70B881F991F5A95A9F78095909540
:1055C000BC01CD010895CF93DF938230910510F493
:1055D00082E090E0E0910A05F0910B0520E030E0D8
:1055E000A0E0B0E0309739F1408151814817590768
:1055F000B8F04817590771F482819381109729F008
:1056000013969C938E9312972CC090930B058093C6
:105610000A0527C02115310531F04217530718F04C
:10562000A901DB0101C0EF019A01BD01DF01028088
:10563000F381E02DD7CF21153105F9F0281B390B67
:105640002430310580F48A819B816115710521F038
:10565000FB019383828304C090930B0580930A051A
:10566000FE01329644C0FE01E20FF31F8193919335
:1056700022503109398328833AC02091080530919E
:105680000905232B41F4209102013091030130934D
:105690000905209308052091000130910101211591
:1056A000310541F42DB73EB74091040150910501F9
:1056B000241B350BE0910805F0910905E217F3076B
:1056C000A0F42E1B3F0B2817390778F0AC014E5F72
:1056D0005F4F2417350748F04E0F5F1F50930905A1
:1056E000409308058193919302C0E0E0F0E0CF0180
:1056F000DF91CF910895CF93DF93009709F487C08E
:10570000FC01329713821282C0910A05D0910B05D9
:10571000209781F420813181280F391F809108055D
:10572000909109058217930779F5F0930905E093A5
:1057300008056DC0DE0120E030E0AE17BF0750F471
:1057400012964D915C9113979D014115510509F1F8
:10575000DA01F3CFB383A28340815181840F951F77
:105760008A179B0771F48D919C911197840F951F57
:1057700002969183808312968D919C9113979383C7
:1057800082832115310529F4F0930B05E0930A0576
:105790003EC0D9011396FC93EE9312974D915D9103
:1057A000A40FB51FEA17FB0779F480819181840F5C
:1057B000951F0296D90111969C938E9382819381B5
:1057C00013969C938E931297E0E0F0E08A819B8180
:1057D000009719F0FE01EC01F9CFCE010296288165
:1057E0003981820F931F20910805309109052817F0
:1057F000390769F4309729F410920B0510920A05C5
:1058000002C013821282D0930905C0930805DF916C
:10581000CF910895A0E0B0E0E0E1FCE20C94C22F4B
:10582000EC01CB01209719F40E94E32AB8C0FE01D5
:10583000E60FF71F9E0122503109E217F30708F423
:10584000ACC0D9010D911C91119706171707B8F03C
:105850000530110508F49FC0A801445051094617AE
:10586000570708F498C002501109061B170B019343
:1058700011936D937C93CF010E947B2B8CC05B01B5
:10588000A01AB10A4E01800E911EA0910A05B09196
:105890000B05612C712C60E070E0109709F449C091
:1058A000A815B905C9F5ED90FC901197670142E084
:1058B000C40ED11CCA14DB0478F147018A189B0876
:1058C000640142E0C40ED11C1296BC90129713964C
:1058D000AC91B5E0CB16D10440F0B282A3839182A3
:1058E0008082D9018D939C9309C00E5F1F4F0E0DCE
:1058F0001F1DF90111830083EB2DFA2F611571052E
:1059000031F0DB011396FC93EE93129744C0F093B1
:105910000B05E0930A053FC06D917C9111976616C7
:10592000770608F43B01BD0112960D90BC91A02DA5
:10593000B4CF609108057091090568157905E9F4FF
:1059400068167906D0F4409100015091010141158B
:10595000510541F44DB75EB76091040170910501A6
:10596000461B570BE417F507C0F4F0930905E093C5
:105970000805F901918380830EC00E94E32A7C010F
:10598000009759F0A801BE010E94D42CCE010E94BC
:105990007B2BC70104C0CE0102C080E090E0CDB7F0
:1059A000DEB7EEE00C94DE2FFB01DC0102C00190BB
:1059B0000D9241505040D8F70895FB01DC01019051
:1059C0000D920020E1F708954532510520F4423050
:1059D00010F00C94EF2CFB011082CB010895BB2733
:1059E0004A3031F4992322F4BDE2909581959F4F7E
:1059F0000C94FB2CBB27FB015527AA27880F991F66
:105A0000AA1FA41710F0A41B83955051B9F7A05DED
:105A1000AA3308F0A95DA193009779F7B111B1936A
:105A20001192CB010C941E2FAEE0B0E0EAE1FDE252
:105A30000C94CC2F0D891E8986E08C831A830983F0
:105A40008FEF9FE79E838D83AE01475E5F4F6F8927
:105A5000788DCE0101960E94362DEF81F885E00FFA
:105A6000F11F10822E96E4E00C94E82FACE0B0E039
:105A7000ECE3FDE20C94BE2F7C016B018A01FC017A
:105A800017821682838181FFBDC1CE0101964C0130
:105A9000F7019381F60193FD859193FF81916F0149
:105AA000882309F4ABC1853239F493FD859193FFC6
:105AB00081916F01853229F4B70190E00E942E2F69
:105AC000E7CF512C312C20E02032A0F48B3269F04A
:105AD00030F4803259F0833269F420612CC08D3269
:105AE00039F0803339F4216026C02260246023C05D
:105AF000286021C027FD27C030ED380F3A3078F4F8
:105B000026FF06C0FAE05F9E300D1124532E13C00D
:105B10008AE0389E300D1124332E20620CC08E3264
:105B200021F426FD6BC1206406C08C3611F4206878
:105B300002C0883641F4F60193FD859193FF81916F
:105B40006F018111C1CF982F9F7D9554933028F418
:105B50000C5F1F4FFFE3F9830DC0833631F08337AD
:105B600071F0833509F05BC022C0F8018081898320
:105B70000E5F1F4F44244394512C540115C038012B
:105B8000F2E06F0E711CF801A080B18026FF03C007
:105B9000652D70E002C06FEF7FEFC5012C870E947A
:105BA000132F2C0183012C852F77222E17C038014B
:105BB000F2E06F0E711CF801A080B18026FF03C0D7
:105BC000652D70E002C06FEF7FEFC5012C870E944A
:105BD000082F2C012C852068222E830123FC1BC05A
:105BE000832D90E048165906B0F4B70180E290E0AA
:105BF0000E942E2F3A94F4CFF50127FC859127FEC1
:105C000081915F01B70190E00E942E2F31103A94EC
:105C1000F1E04F1A51084114510471F7E5C0843680
:105C200011F0893639F5F80127FF07C060817181CD
:105C3000828193810C5F1F4F08C06081718188272A
:105C400077FD8095982F0E5F1F4F2F76B22E97FF0E
:105C500009C090958095709561957F4F8F4F9F4FAC
:105C60002068B22E2AE030E0A4010E94602FA82E06
:105C7000A81844C0853729F42F7EB22E2AE030E0E0
:105C800025C0F22FF97FBF2E8F36C1F018F488356A
:105C900079F0B4C0803719F0883721F0AFC02F2FCA
:105CA0002061B22EB4FE0DC08B2D8460B82E09C0C9
:105CB00024FF0AC09F2F9660B92E06C028E030E06E
:105CC00005C020E130E002C020E132E0F801B7FE7B
:105CD00007C060817181828193810C5F1F4F06C074
:105CE0006081718180E090E00E5F1F4FA4010E94EF
:105CF000602FA82EA818FB2DFF77BF2EB6FE0BC075
:105D00002B2D2E7FA51450F4B4FE0AC0B2FC08C09F
:105D10002B2D2E7E05C07A2C2B2D03C07A2C01C092
:105D2000752C24FF0DC0FE01EA0DF11D808180332A
:105D300011F4297E09C022FF06C07394739404C035
:105D4000822F867809F0739423FD13C020FF06C0CC
:105D50005A2C731418F4530C5718732C731468F4DA
:105D6000B70180E290E02C870E942E2F73942C853F
:105D7000F5CF731410F4371801C0312C24FF12C072
:105D8000B70180E390E02C870E942E2F2C8522FF04
:105D900017C021FF03C088E590E002C088E790E0CB
:105DA000B7010CC0822F867859F021FD02C080E235
:105DB00001C08BE227FD8DE2B70190E00E942E2FFB
:105DC000A51438F4B70180E390E00E942E2F5A9476
:105DD000F7CFAA94F401EA0DF11D8081B70190E09C
:105DE0000E942E2FA110F5CF332009F451CEB70118
:105DF00080E290E00E942E2F3A94F6CFF701868140
:105E0000978102C08FEF9FEF2C96E2E10C94DA2F7E
:105E1000FC010590615070400110D8F78095909575
:105E20008E0F9F1F0895FC0161507040019001107A
:105E3000D8F7809590958E0F9F1F0895DC01FC0187
:105E4000672F71917723E1F7329704C07C916D93AE
:105E500070836291AE17BF07C8F308950F931F9325
:105E6000CF93DF93182F092FEB018B8181FD03C0A6
:105E70008FEF9FEF20C082FF10C04E815F812C8189
:105E80003D81421753077CF4E881F9819F012F5F20
:105E90003F4F39832883108306C0E885F985812F19
:105EA0000995892B29F72E813F812F5F3F4F3F8333
:105EB0002E83812F902FDF91CF911F910F91089505
:105EC000FA01AA27283051F1203181F1E8946F932B
:105ED0006E7F6E5F7F4F8F4F9F4FAF4FB1E03ED0D1
:105EE000B4E03CD0670F781F891F9A1FA11D680F6F
:105EF000791F8A1F911DA11D6A0F711D811D911DA2
:105F0000A11D20D009F468943F912AE0269F112416
:105F10003019305D3193DEF6CF010895462F47707A
:105F2000405D4193B3E00FD0C9F7F6CF462F4F70D5
:105F3000405D4A3318F0495D31FD4052419302D033
:105F4000A9F7EACFB4E0A6959795879577956795D9
:105F5000BA95C9F700976105710508959B01AC01D9
:105F60000A2E06945795479537952795BA95C9F700
:105F7000620F731F841F951FA01D08952F923F92DB
:105F80004F925F926F927F928F929F92AF92BF9249
:105F9000CF92DF92EF92FF920F931F93CF93DF93F5
:105FA000CDB7DEB7CA1BDB0B0FB6F894DEBF0FBE52
:105FB000CDBF09942A88398848885F846E847D849F
:105FC0008C849B84AA84B984C884DF80EE80FD80A1
:105FD0000C811B81AA81B981CE0FD11D0FB6F89417
:0E5FE000DEBF0FBECDBFED010895F894FFCFD8
:105FEE0000000C05800003CC3F0D00594300000A51
:105FFE005B004C6143726F7373654954506C7573DB
:10600E005265616465720031302E316A00202800BD
:10601E0029002040004175746F546F67676C6520CE
:10602E0000205365636F6E647300206B62707300A3
:10603E00202F2000206B487A002A2A2A204C614308
:10604E00726F7373652077656174686572207374FF
:10605E006174696F6E20776972656C6573732072F7
:10606E006563656976657220666F722049542B20D0
:10607E0073656E736F7273202A2A2A0052616469E7
:10608E006F20736574757020636F6D706C657465C9
:10609E002E205374617274696E6720746F2072655E
:1060AE006365697665206D65737361676573000A54
:1060BE00456E6420726563656976696E672C20484B
:1060CE0045582072617720646174613A20005265F0
:1060DE006C6179656400253036642000454D543777
:1060EE00313130205B005D00204352433A57524F0E
:1060FE004E4700204352433A4F4B0020533A002064
:10610E0049443A0020563A00206D413A0020573A51
:10611E0000206B57683A0020436F6E2E3A002050D5
:10612E006169723A00204352433A004F4B20454D6D
:10613E00543731313020004F4B20392000204E652E
:10614E0077426174743A002042697431323A002009
:10615E0054656D703A00205765616B426174743AF4
:10616E00002048756D3A004C6143726F7373652061
:10617E005B00232320435243204641494C202323D6
:10618E00004E6F2076616C696420737461727400C6
:10619E004E6F2076616C69642054656D7065726116
:1061AE00747572653A20004E6F2076616C696420BA
:1061BE004C6576656C3A20004E6F2076616C696492
:1061CE0020566F6C746167653A20004C6576656C7D
:1061DE0053656E646572205B00204C6576656C3A83
:1061EE000020566F6C743A004F4B204C5320002009
:1061FE0030200052464D3132420052464D36394320
:10620E0057004E6F6E6500526164696F2069733A74
:10621E00200053656E64696E6720646174613A2074
:10622E00004F4B2057532000203100545832324932
:10623E0054205B00204C6F77426174743A00204505
:10624E0072726F723A002D2D2D00205261696E3AD6
:10625E00002057696E643A002066726F6D3A002016
:10626E00477573743A00206D2F73005458333849B4
:10627E0054205B0000000000C5224124472260220A
:10628E005222A3226E616E00696E66006F76660002
:02629E002E00D0
:00000001FF
